:0400000019C070C0F3
:10000400FDCFFCCFFBCFFACF83C0F8CFF7CFF6CF2D
:10001400083E11122642400E000280FF84E0C97798
:100024000000100076001400010004002400000009
:10003400F894EE27ECBBE5BFF8E1A4B7A77FA4BF13
:10004400F1BDE1BD8DE0A2E0ED938A95E9F780E48E
:10005400A0E6ED938A95E9F7E6E2F0E0C8953196DB
:10006400802DC8953196902D0097B9F0C89531969A
:10007400A02DC8953196B02DC8953196102CC895F1
:1000840031966E2F7F2FF02DE12DC89531960D926C
:100094000197D9F7E62FF72FE1CFEFE9EDBFC6E7D8
:1000A4009EC0AA932DD110E0EB811E17A0F400E8A6
:1000B40020E0283070F4E12FAC81AE0FEC91E02306
:1000C40011F0C39A01C0C398C29AC29806952F5FD3
:1000D400F0CF1F5FE9CFC09AC09816D12596089536
:1000E400AA93EA93EFB7EA93E0918700EF5FE09376
:1000F4008700A0918700A93118F0E8E1E093870018
:10010400E0E0E0938B00E991EFBFE991A9911895A4
:100114000A921A92FA926A937A938A939A93AA9376
:10012400BA93EA93FA93EFB7EA93E0918B00EF5F07
:10013400E0938B00A0918B00AF3F19F4E0E0E093D3
:100144008900E0918A00EF5FE0938A00A0918A0021
:10015400A130B1F4E0918900E03019F4E091850018
:1001640008C0A0918900BB27EAE0F0E0ACD0EA58CF
:10017400E081E0938600E6E8EA93A1E092DFC49888
:10018400A0918A00A230E9F4A0918900AA3030F449
:10019400E0918100E058E09386000CC0A0918900B2
:1001A400B0E0EAE0F0E08AD0EA58E081E058E09379
:1001B4008600C49AE0E0E0938A00E6E8EA93A1E0CE
:1001C40070DFE991EFBFF991E991B991A991999102
:1001D400899179916991F990199009901895E0E8BD
:1001E400E6BDE0E0E6BDE0E2E8BBEDE1E7BBE0E46C
:1001F400EBBFE3E0E5BFE0E4EABFE2E0EFBDE5E04A
:10020400E3BFE0E0E2BFE2E3E6BFE0E0E9BDE4E053
:10021400E9BFE0918000E0938600E6E8EA93A1E07C
:1002240040DFC498A0EDB7E026D07894A3E0B0E016
:1002340022D0A0918700A13030F0E0918800A091F5
:100244008700EA1709F011C0E0E0E0938700E0912D
:100254008800E0938900E42DE457A0918800A083EE
:100264004394E3E0E41508F44424E0918700E09328
:100274008800DCCFFFCF109639F080EB94E0019733
:10028400F1F7A8951197C9F70895F195E195F04014
:1002940008950024112490E1AA0FBB1F001C111C17
:1002A4000E1A1F0A18F40E0E1F1E01C0A1609A95A3
:1002B40099F7EA2FFB2FA02DB12D089513D0E9DF74
:1002C4000EF4E3DF0895E894B7FF04C0A095B09559
:1002D40011966894F7FDD9DFDCDFEA2FFB2F0EF4CB
:1002E400D4DF0895E894F7FF02C0CFDF6894B7FF26
:1002F40006C0A095B095119600F8039400FA0895ED
:100304002A931A930A9308952A81198108810895DA
:00000001FF
